:020000000134C9
:20003400758171758901D2AFD28C1204C212001B80FB0581740A75F000C0E0C0F074027543
:20005400F000C0E0C0F01207BF15811581158115815480C5F05400C5F078FE122866F64539
:20007400F07003020098E61228987BFF12288F12299945F0700302009574FF75F0FF020088
:200094009D020048740175F000158122120046740A75F000C0E0C0F0740075F000C0E0C00F
:2000B400F0740175F000C0E0C0F01207E87FFA122872221200467BFF7CFF12299945F07004
:2000D400030200E074FF75F0FF020149740A75F000C0E0C0F0740075F000C0E0C0F07438FC
:2000F40075F000C0E0C0F01207E87FFA122872120046740A75F000C0E0C0F0740075F000AD
:20011400C0E0C0F0740C75F000C0E0C0F01207E87FFA1228721200A0740075F000C0E0C035
:20013400F0740075F000C0E0C0F012014A15811581158115812212004678FB122866E61258
:20015400289890020C0228A1740A75F000C0E0C0F0740075F000C0E0C0F078F5122866E613
:200174002480122898C0E0C0F01207E87FFA122872020220740A75F000C0E0C0F07400753F
:20019400F000C0E0C0F078F5122866E624C0122898C0E0C0F01207E87FFA122872020220C8
:2001B400740A75F000C0E0C0F0740075F000C0E0C0F078F5122866E62494122898C0E0C0F2
:2001D400F01207E87FFA122872020220740A75F000C0E0C0F0740075F000C0E0C0F078F508
:2001F400122866E624D4122898C0E0C0F01207E87FFA122872020220E0010300B401020066
:20021400880101005C01000000002002220581740078FE122866F678FE122866E618181855
:2002340018860108860275F00012288889828A83E4931228987B0012288F1229A245F0702D
:20025400030202A7800B78FE122866E604F61480C6120046740A75F000C0E0C0F07401758C
:20027400F000C0E0C0F078FA122866E618181818860108860275F00012288889828A83E498
:2002940093122898C0E0C0F01207E87FFA12287202025A78FA122866E60886F015812212D1
:2002B4000046740A75F000C0E0C0F0740175F000C0E0C0F078F7122866E6122898C0E0C060
:2002D400F01207E87FFA122872227F0812287278F3122866E60886F07B007C001229794540
:2002F400F0700302030D740075F00079F712286B122888742DF702031D740075F00079F7C2
:2003140012286B122888742BF778F3122866E60886F078FD122866F608A6F078F3122866A9
:20033400E60886F07B007C0012297945F0700302036B78FD122866E60886F012297278F3F1
:20035400122866F608A6F018E60886F012295F18F608A6F0122968740175F00079F712286C
:200374006B12288878F3122866E60886F07BE87C031228E52430C5F03400C5F0F718E608DD
:2003940086F07BE87C031228DE78FD122866F608A6F0740275F00079F712286B1228887806
:2003B400FD122866E60886F07B647C001228E52430C5F03400C5F0F778F3122866E6088646
:2003D400F07B647C001228DE78FD122866F608A6F0740375F00079F712286B12288878FDD5
:2003F400122866E60886F07B0A7C001228E52430C5F03400C5F0F7740475F00079F7122855
:200414006B12288878FD122866E60886F07B0A7C001228DE2430C5F03400C5F0F774007537
:20043400F00079F712286B122888E7122898C0E0C0F01202B315811581740175F00079F79B
:2004540012286B122888E7122898C0E0C0F01202B315811581740275F00079F712286B1223
:200474002888E7122898C0E0C0F01202B315811581740375F00079F712286B122888E71210
:200494002898C0E0C0F01202B315811581740475F00079F712286B122888E7122898C0E038
:2004B400C0F01202B3158115817FF8022881758E037481F5A8E5884401F5887400F53A7485
:2004D40000F56C740C75F000C0E0C0F0740075F000C0E0C0F0E53A122898C0E0C0F01207EF
:2004F400E87FFA1228727400F511747075F017F55D85F05E746475F000F55385F0547963B2
:200514007A00E98AF0C0E0C0F0746475F000C0E0C0F012266B15811581158115811219CA1D
:200534001200C7749975F02DC0E0C0F012022115811581740075F000C0E0C0F0740175F07B
:2005540000C0E0C0F012014A158115811581158174A275F02DC0E0C0F01202211581158129
:2005740074E875F003C0E0C0F012269E1581158174BFF537E5114402F5111215CF74807551
:20059400F025C0E0C0F01226BB1581158179017A2AE98AF0C0E0C0F01226DE15811581129E
:2005B400110A1211FD12116C1210E9120FC21209B2120EED120C7B120CF3120D301212CFA9
:2005D4001214FA1216A5121ACF1218A8121B66121B8F121C4D121EB2122289120989121519
:1705F4003312159D1215CF12077B120F9912237C1223F00205B62200
:07000300C0D0C0E002060BB3
:20060B00C0F0C083C082C000C001C002C003C004C005C006C00712063FD007D006D005D0D5
:20062B0004D003D002D001D000D082D083D0F0D0E0D0D032740875F000C0E0C0F074027562
:20064B00F000C0E0C0F01207BF1581158115811581F53D85F03E740875F000C0E0C0F07495
:20066B000175F000C0E0C0F01207BF1581158115811581F53F85F040E53F8540F05410C59E
:20068B00F05400C5F0F53BE53F8540F05420C5F05400C5F0F53CE53F8540F0540FC5F054A5
:2006AB0000C5F0F53F85F040E53F8540F07B087C00122940F53F85F040E53D853EF0453FFC
:2006CB00C5F04540C5F0F53D85F03EE53B60030206EEE53D853EF07BFF7CFF1228CAF53DC2
:2006EB0085F03EE53C70030206FF740F75F027F53D85F03EE53A122898C333C5F033C5F029
:20070B0079437A00122888E53D853EF0F709A7F0E53A04F53A14E53A5403F53A740C75F07A
:20072B0000C0E0C0F0740075F000C0E0C0F0E53A122898C0E0C0F01207E87FFA122872745A
:20074B000175F000C0E0C0F012269E15811581E53A1228987B0012288F12299945F0700325
:20076B0002077AE59054BFF590E5114480F51122E51675F0007B627C0012299945F07003C7
:20078B000207A379147A2DE98AF0C0E0C0F01226DE1581158112110A2278FB122866E6F53C
:2007AB0013E513A2E09290A2E19291A2E29292A2E392932278F9122866E6122898C0E0C03C
:2007CB00F01207A41581158178FB122866E60886F0C0E0C0F012271A158115812278F7124C
:2007EB002866E6122898C0E0C0F01207A41581158178F9122866E60886F0C0E0C0F008E6BC
:20080B00122898C0E0C0F012273B15811581158115812212275B74D075F000C0E0C0F0121E
:20082B00277015811581740775F000C0E0C0F012277015811581749075F000C0E0C0F0121A
:20084B002770158115811227682212275B74D075F000C0E0C0F012277015811581740075BC
:20086B00F000C0E0C0F01227701581158112276812275B74D175F000C0E0C0F0122770156B
:20088B008115817400F5717400F515E51575F0007B067C001229AC45F070030208CE800893
:2008AB00E51504F5151480E3E515794B7A0075F000122888C001C00212279AD007D000F65C
:2008CB000208AB7401F571E515794B7A0075F000122888C001C00212279AD007D000F61219
:2008EB0027682212275B74D075F000C0E0C0F012277015811581740075F000C0E0C0F0129F
:20090B00277015811581740075F000C0E0C0F012277015811581743075F000C0E0C0F012A0
:20092B00277015811581741275F000C0E0C0F012277015811581740375F000C0E0C0F0129B
:20094B00277015811581742575F000C0E0C0F012277015811581740775F000C0E0C0F01264
:20096B00277015811581740075F000C0E0C0F0122770158115811227682212085522E5165C
:20098B0075F0007B757C0012299945F070030209B179317A2CE98AF0C0E0C0F01226DE1515
:2009AB0081158112110A22E51675F0007B747C0012299945F07003020A5D74AA75F02DC0A6
:2009CB00E0C0F01226DE15811581120B14F50D743A75F000C0E0C0F01226F215811581123C
:2009EB000B14F50C743A75F000C0E0C0F01226F215811581120B14F50A12275B74D075F0A6
:200A0B0000C0E0C0F012277015811581740075F000C0E0C0F012277015811581E50A75F054
:200A2B0000C0E0C0F012277015811581E50C75F000C0E0C0F012277015811581E50D75F0B4
:200A4B0000C0E0C0F01227701581158112276812110A227F09122872740075F00078FD12E2
:200A6B002866F608A6F012270AC0E0C0F01226F21581158178FC122866F67B0D7C00122917
:200A8B00A245F07003020AC6801678FD122866E60886F012295F18F608A6F012296880C6F1
:200AAB0078FD122866E60886F079F612286B12288878FC122866E6F7020A9578FD12286635
:200ACB00E60886F079F612286B1228887400F778FD122866E60886F07B007C0012299945DD
:200AEB00F07003020AF974FF75F0FF020B0F79F612286BE98AF0C0E0C0F01227CE15811517
:200B0B0081020B0F7FF702288105810581058105810581740075F00078FD122866F608A6DC
:200B2B00F078FD122866E60886F07B027C0012297945F07003020B86801678FD122866E6C8
:200B4B000886F012295F18F608A6F012296880D178FD122866E60886F079FA12286B122807
:200B6B0088C001C00212270AC0E0C0F01226F215811581D007D000F6020B4578FD12286672
:200B8B00E60886F079FA12286B1228887400F7740075F00079FA12286B122888E7C3943080
:200BAB001228987B0412288F122940C0E0C0F0740175F00079F812286B122888E7C3943025
:200BCB00D004D0034BC5F04CC5F01228987FFB02288105810581058105810581740075F0F4
:200BEB000078FD122866F608A6F078FD122866E60886F07B027C0012297945F07003020C65
:200C0B004F801678FD122866E60886F012295F18F608A6F012296880D178FD122866E6082E
:200C2B0086F079FA12286B122888C001C00212270AC0E0C0F01226F215811581D007D00046
:200C4B00F6020C0E78FD122866E60886F079FA12286B1228887400F779FA12286BE98AF03E
:200C6B00C0E0C0F01227CE158115817FFB022881E51675F0007B697C0012299945F0700385
:200C8B00020CF274C975F02DC0E0C0F01226DE15811581740075F000C0E0C0F01207A415ED
:200CAB00811581740475F000C0E0C0F0120A5E7B647C001228CAC0E0C0F01227491581158F
:200CCB008115811581740475F000C0E0C0F012272915811581F55D85F05EE55D855EF0F572
:200CEB005B85F05C12110A22E51154087003020D2FE55B855CF0122968F55B85F05C12295B
:200D0B005FE55B855CF07B007C001229B345F07003020D2FE55D855EF0F55B85F05CE51161
:200D2B004404F511220581E51714F51704E51775F0007B007C001229B345F07003020EEAAA
:200D4B007464F517120855740275F000794B7A00122888E775F0007B047C0012294E78FE14
:200D6B00122866F6E675F0007B0A7C001228CAF6740275F000794B7A00122888C001C0022E
:200D8B00740275F000794B7A00122888E7540F78FC12286626D007D000F6740175F00079F9
:200DAB004B7A00122888E775F0007B047C0012294E78FE122866F6E675F0007B0A7C001267
:200DCB0028CAF6740175F000794B7A00122888C001C002740175F000794B7A00122888E702
:200DEB00540F78FC12286626D007D000F6740075F000C0E0C0F01207A415811581740275B1
:200E0B00F000794B7A00122888C001C002740075F000C0E0C0F012271A15811581D007D005
:200E2B000086037C0012299945F0602B740175F000794B7A00122888C001C002740175F0D7
:200E4B0000C0E0C0F012271A15811581D007D00086037C0012299945F07003020E79E51111
:200E6B004408F511742C75F001F55385F054740275F000794B7A00122888C001C00274022A
:200E8B0075F000C0E0C0F012271A15811581D007D00086037C0012299945F0602B740175E9
:200EAB00F000794B7A00122888C001C002740375F000C0E0C0F012271A15811581D007D062
:200ECB000086037C0012299945F07003020EEAE51154F7F511746475F000F55385F05415E2
:200EEB008122E51675F0007B647C0012299945F07003020F9874E175F02DC0E0C0F01226F5
:200F0B00DE15811581120B14F50E742D75F000C0E0C0F01226F215811581120B14F50F7433
:200F2B002D75F000C0E0C0F01226F215811581120B14F51012275B74D075F000C0E0C0F0AB
:200F4B0012277015811581740475F000C0E0C0F012277015811581E50E75F000C0E0C0F007
:200F6B0012277015811581E50F75F000C0E0C0F012277015811581E51075F000C0E0C0F069
:200F8B001227701581158112276812110A22E51675F0007B0D7C0012299945F07003020F90
:200FAB00C179017A2AE98AF0C0E0C0F01226DE1581158112110A22E51675F0007B2F7C007D
:200FCB0012299945F070030210E8120855740075F02EC0E0C0F0740475F000794B7A00129D
:200FEB002888E775F000C0E0C0F0740575F000794B7A00122888E775F000C0E0C0F07406A6
:20100B0075F000794B7A00122888E775F000C0E0C0F0740475F0001224277FF812287274F3
:20102B001175F02EC0E0C0F0740275F000794B7A00122888E775F000C0E0C0F0740175F060
:20104B0000794B7A00122888E775F000C0E0C0F0740075F000794B7A00122888E775F000C4
:20106B00C0E0C0F0740475F0001224277FF81228721211D8742175F02EC0E0C0F07400755C
:20108B00F00079437A00122888E70987F0C0E0C0F0740275F00079437A00122888E709875C
:2010AB00F0C0E0C0F0740475F00079437A00122888E70987F0C0E0C0F0740675F0007943BE
:2010CB007A00122888E70987F0C0E0C0F0740575F0001224277FF612287212110A22E598EA
:2010EB005401700302110512270AC0E0C0F01226F215811581F51602110974FFF5162279DC
:20110B001C7A2AE98AF0C0E0C0F01226DE158115812205810581740075F00078FD122866F3
:20112B00F608A6F078FD122866E60886F078F9122866860308860412297945F070030211FC
:20114B0067801678FD122866E60886F012295F18F608A6F012296880CB02114E158115814D
:20116B00221211731211AD22E559855AF012295FF55985F05A122968E559855AF0AB53AC9C
:20118B00541229BC45F070030211AC740075F000F55985F05AE5114440F511C2977405F555
:2011AB001422E511544070030211D7E51414F51404E51475F0007B007C0012299945F0701F
:2011CB00030211D7D297E51154BFF51122E5904440F590E511548075F0007B007C0012299E
:2011EB009945F070030211F60211DEE511547FF51122308DFDC28D438CDC22058105817462
:20120B000175F00079637A00122888E775F00078FD122866F608A6F018E60886F07B087CD5
:20122B000012294018F608A6F0740075F00079637A0012288878FD122866E60886F04715B6
:20124B008115812274012563F563E43564F564E43565F5652212124F740275F00079637A81
:20126B0000122888E775F000C0E0C0F01207A4158115811212062212124F12124F740275FF
:20128B00F00079637A00122888E775F000C0E0C0F01207A4158115811212062278FB1228BD
:2012AB0066E675F0007B047C0012294EF62430C5F03400C5F02278FB122866E6540F243034
:2012CB0012289822E511540470030214B81211D8120855121282C0E0C0F0E5578558F0C057
:2012EB00E0C0F01227491581158115811581121260C0E0C0F0740475F000794B7A00122850
:20130B0088E775F000C0E0C0F012273B1581158115811581121260C0E0C0F0740575F00020
:20132B00794B7A00122888E775F000C0E0C0F012273B1581158115811581121260C0E0C056
:20134B00F0740675F000794B7A00122888E775F000C0E0C0F012273B15811581158115814B
:20136B00121260C0E0C0F0740275F000794B7A00122888E775F000C0E0C0F012273B15810D
:20138B00158115811581121260C0E0C0F0740175F000794B7A00122888E775F000C0E0C026
:2013AB00F012273B1581158115811581121260C0E0C0F0740075F000794B7A00122888E7D2
:2013CB0075F000C0E0C0F012273B1581158115811581121282C0E0C0F0740075F0007943F6
:2013EB007A00122888E70987F0C0E0C0F01227491581158115811581121282C0E0C0F074AB
:20140B000275F00079437A00122888E70987F0C0E0C0F012274915811581158115811212AD
:20142B0082C0E0C0F0740475F00079437A00122888E70987F0C0E0C0F01227491581158195
:20144B0015811581121282C0E0C0F0740675F00079437A00122888E70987F0C0E0C0F012BF
:20146B0027491581158115811581E51154FBF511E5578558F012295FF55785F0581214B9B3
:20148B00740075F000C0E0C0F01207A415811581740675F000C0E0C0F0E5578558F0C0E057
:2014AB00C0F0122749158115811581158122E5578558F07B887C131229BC45F07003021425
:2014CB00F9E51154F7F511746475F000F55385F054743C75F000C0E0C0F074FF75F0FFC077
:2014EB00E0C0F012273B158115811581158122E51675F0007B727C0012299945F07003021C
:20150B001532742E75F02EC0E0C0F0E5578558F0C0E0C0F0740275F0001224271581158137
:20152B001581158112110A22740E75F000C0E0C0F0740075F000C0E0C0F01207BF15811542
:20154B0081158115817BFF7C001229A245F0600EE511540175F0007B007C0012299945F0AD
:20156B007003021598E5114401F511740E75F000C0E0C0F0740075F000C0E0C0F01207BFC5
:20158B001581158115811581F53702159C74FFF53722740E75F000C0E0C0F0740075F00038
:2015AB00C0E0C0F01207BF15811581158115817BFF7C0012299945F070030215CEE51154FF
:2015CB00FEF51122E53775F0007BFF7C001229A245F070030216A4E53775F0009016900269
:2015EB0028A1E56C04F56C140216A4E5116402F511E51154EFF5111200A0740075F000C0A5
:20160B00E0C0F0740175F000C0E0C0F012014A1581158115811581744475F02EC0E0C0F0B5
:20162B0012022115811581E5115402700302164E742A75F000C0E0C0F01202B315811581D3
:20164B000216871200A01222F0740075F000C0E0C0F0740075F000C0E0C0F012014A1581C5
:20166B00158115811581744C75F02EC0E0C0F012022115811581E5114410F5110216A4028B
:20168B0016A40216A48D16EF008A16DF00F615BF00ED157F000000A41622E51675F0007BB6
:2016AB00737C0012299945F0700302184B740075F000C0E0C0F01207A415811581745575FF
:2016CB00F02EC0E0C0F0740075F000C0E0C0F012271A15811581C0E0C0F0740175F000C0FF
:2016EB00E0C0F012271A15811581C0E0C0F0740375F0001224277FFA122872740075F00049
:20170B00C0E0C0F0120BDD122898C0E0C0F012273B1581158115811581743A75F000C0E0D3
:20172B00C0F01226F215811581740175F000C0E0C0F0120BDD122898C0E0C0F012273B15C9
:20174B0081158115811581746875F02EC0E0C0F0740275F000C0E0C0F012271A15811581D2
:20176B00C0E0C0F0740375F000C0E0C0F012271A15811581C0E0C0F0740375F000122427DA
:20178B007FFA122872740275F000C0E0C0F0120BDD122898C0E0C0F012273B15811581151D
:2017AB00811581743A75F000C0E0C0F01226F215811581740375F000C0E0C0F0120BDD1216
:2017CB002898C0E0C0F012273B1581158115811581747B75F02EC0E0C0F0740075F000C0B7
:2017EB00E0C0F012271A15811581C0E0C0F0740175F000C0E0C0F012271A15811581C0E036
:20180B00C0F0740275F000C0E0C0F012271A15811581C0E0C0F0740375F000C0E0C0F012D5
:20182B00271A15811581C0E0C0F0740575F0001224277FF612287212184C1222F012110ABD
:20184B0022740075F000C0E0C0F012271A158115817B637C0012299945F0700302188A74C5
:20186B003C75F000C0E0C0F0740175F000C0E0C0F012273B15811581158115810218A77441
:20188B003C75F000C0E0C0F074FF75F0FFC0E0C0F012273B158115811581158122E51675C7
:2018AB00F0007B3D7C0012299945F070030219C9740075F000C0E0C0F01207A41581158187
:2018CB00749175F02EC0E0C0F0740075F000C0E0C0F012271A15811581C0E0C0F074017533
:2018EB00F000C0E0C0F012271A15811581C0E0C0F0740375F0001224277FFA12287274A359
:20190B0075F02EC0E0C0F0740275F000C0E0C0F012271A15811581C0E0C0F0740375F00003
:20192B00C0E0C0F012271A15811581C0E0C0F0740375F0001224277FFA12287274B575F091
:20194B002EC0E0C0F0740475F000C0E0C0F0122729158115817B647C001228E5C0E0C0F079
:20196B00740275F0001224271581158115811581743C75F000C0E0C0F012271A15811581E8
:20198B007B017C0012299945F070030219B174D375F02EC0E0C0F0740175F0001224271586
:2019AB008115810219C674DC75F02EC0E0C0F0740175F0001224271581158112110A2274CB
:2019CB000075F000C0E0C0F01207A415811581740475F000C0E0C0F012272915811581F5AE
:2019EB005D85F05EE55D855EF0F55B85F05C740675F000C0E0C0F012272915811581F5576D
:201A0B0085F05879697A00E98AF0C0E0C0F0742E75F000C0E0C0F012266B15811581158123
:201A2B00158179667A00E98AF0C0E0C0F0E5578558F0C0E0C0F012266B1581158115811526
:201A4B008179667A00E98AF0C0E0C0F079697A00E98AF0C0E0C0F01225BD15811581158129
:201A6B00158179667A00E98AF0C0E0C0F0746475F000C0E0C0F012266B15811581158115B2
:201A8B0081796D7A00E98AF0C0E0C0F079667A00E98AF0C0E0C0F012257C15811581158126
:201AAB00158179637A00E98AF0C0E0C0F0796D7A00E98AF0C0E0C0F012262E1581158115C2
:201ACB0081158122E51675F0007B6E7C0012299945F07003021B6574E375F02EC0E0C0F0C5
:201AEB001226DE1581158112270A7B797C0012299945F07003021B62E51154F7F511740030
:201B0B0075F000F55785F058740075F000C0E0C0F01207A415811581740675F000C0E0C0EB
:201B2B00F0740075F000C0E0C0F0122749158115811581158179637A00E98AF0C0E0C0F09E
:201B4B00746475F000C0E0C0F012266B158115811581158112211F12110A22E51675F000F1
:201B6B007B3F7C0012299945F07003021B8E79207A2AE98AF0C0E0C0F01226DE15811581CB
:201B8B0012110A22E51675F0007B637C0012299945F07003021C4C12085574F675F02EC01F
:201BAB00E0C0F0740475F000794B7A00122888E775F000C0E0C0F0740575F000794B7A00F5
:201BCB00122888E775F000C0E0C0F0740675F000794B7A00122888E775F000C0E0C0F074AD
:201BEB000475F0001224277FF8122872740775F02FC0E0C0F0740275F000794B7A0012283F
:201C0B0088E775F000C0E0C0F0740175F000794B7A00122888E775F000C0E0C0F074007536
:201C2B00F000794B7A00122888E775F000C0E0C0F0740475F0001224277FF812287212118D
:201C4B000A22E51675F0007B617C0012299945F07003021EB11221F379667A00E98AF0C0A6
:201C6B00E0C0F0740175F000C0E0C0F012266B158115811581158179637A00E98AF0C0E04B
:201C8B00C0F079667A00E98AF0C0E0C0F012258F158115811581158179667A00E98AF0C0E3
:201CAB00E0C0F079637A00E98AF0C0E0C0F012262E158115811581158179637A00E98AF009
:201CCB00C0E0C0F0746475F000C0E0C0F012266B1581158115811581740075F000F561856D
:201CEB00F062E5618562F0AB57AC581229AC45F07003021EAE8012E5618562F012295FF5C9
:201D0B006185F06212296880D9740D75F000C0E0C0F012210D15811581740A75F000C0E05F
:201D2B00C0F012210D15811581121282C0E0C0F012272915811581741775F02FC0E0C0F089
:201D4B00E5618562F0C0E0C0F0740275F0001224271581158115811581741B75F02FC0E0B8
:201D6B00C0F0121260C0E0C0F012271A15811581C0E0C0F0121260C0E0C0F012271A158148
:201D8B001581C0E0C0F0121260C0E0C0F012271A15811581C0E0C0F0740475F00012242775
:201DAB007FF8122872742B75F02FC0E0C0F0121260C0E0C0F012271A15811581C0E0C0F0CF
:201DCB00121260C0E0C0F012271A15811581C0E0C0F0121260C0E0C0F012271A1581158102
:201DEB00C0E0C0F0740475F0001224277FF8122872743B75F02FC0E0C0F0121282C0E0C092
:201E0B00F012272915811581C0E0C0F0740275F0001224271581158115811581743F75F041
:201E2B002FC0E0C0F0121282C0E0C0F012272915811581C0E0C0F0740275F00012242715F7
:201E4B0081158115811581744375F02FC0E0C0F0121282C0E0C0F012272915811581C0E075
:201E6B00C0F0740275F0001224271581158115811581744775F02FC0E0C0F0121282C0E032
:201E8B00C0F012272915811581C0E0C0F0740275F00012242715811581158115811220D314
:201EAB00021D0212110A22E51675F0007B787C0012299945F070030220D21221F379667AE9
:201ECB0000E98AF0C0E0C0F0740175F000C0E0C0F012266B158115811581158179637A00C9
:201EEB00E98AF0C0E0C0F079667A00E98AF0C0E0C0F012258F158115811581158179667AA1
:201F0B0000E98AF0C0E0C0F079637A00E98AF0C0E0C0F012262E1581158115811581796360
:201F2B007A00E98AF0C0E0C0F0746475F000C0E0C0F012266B1581158115811581740075F8
:201F4B00F000F56185F062E5618562F0AB57AC581229AC45F070030220CF8012E5618562F7
:201F6B00F012295FF56185F06212296880D9740D75F000C0E0C0F012210D15811581740A83
:201F8B0075F000C0E0C0F012210D15811581121282C0E0C0F012272915811581744B75F06D
:201FAB002FC0E0C0F0E5618562F0C0E0C0F0740275F0001224271581158115811581121276
:201FCB0060C0E0C0F012271A15811581121260C0E0C0F012271A15811581121260C0E0C090
:201FEB00F012271A15811581121260C0E0C0F012271A15811581121260C0E0C0F012271AED
:20200B0015811581121260C0E0C0F012271A15811581744F75F02FC0E0C0F0121282C0E049
:20202B00C0F012272915811581C0E0C0F0740275F00012242715811581158115817453753B
:20204B00F02FC0E0C0F0121282C0E0C0F012272915811581C0E0C0F0740275F000122427FA
:20206B001581158115811581745775F02FC0E0C0F0121282C0E0C0F012272915811581C00A
:20208B00E0C0F0740275F0001224271581158115811581745B75F02FC0E0C0F0121282C0FC
:2020AB00E0C0F012272915811581C0E0C0F0740275F00012242715811581158115811220E5
:2020CB00D3021F6712110A2205811228127B137C0012299945F0700302210A78FE122866B0
:2020EB00E61228987B1112288F1229A245F0700302210A12281278FE122866F60220E615A1
:20210B00812278FB122866E6F5133099FDC299E513F59922745F75F02FC0E0C0F01226DE7A
:20212B001581158179187A00E98AF0C0E0C0F0741E75F000C0E0C0F01228241581158115C4
:20214B00811581740075F000C0E0C0F01207A415811581740075F000F56185F062E561857A
:20216B0062F079187A00122888E775F0007B007C001229A245F070030221CD8012E5618520
:20218B0062F012295FF56185F06212296880CEE5618562F02408C5F03400C5F0C0E0C0F0F3
:2021AB00E5618562F079187A00122888E775F000C0E0C0F012273B158115811581158102C0
:2021CB002188E5618562F02408C5F03400C5F0C0E0C0F0740075F000C0E0C0F012273B1562
:2021EB0081158115811581220581740D75F000C0E0C0F012210D15811581740A75F000C0A4
:20220B00E0C0F012210D15811581740075F000C0E0C0F01207A415811581740075F000F5D7
:20222B006185F062E5618562F02408C5F03400C5F0C0E0C0F012271A1581158178FE1228F5
:20224B0066F67B007C001229A245F070030222868012E5618562F012295FF56185F0621269
:20226B00296880C078FE122866E6122898C0E0C0F01226F21581158102225D158122740061
:20228B0075F000C0E0C0F01207A415811581743C75F000C0E0C0F012271A158115817B0135
:2022AB007C0012299945F070030222EFE5B0540875F0007B007C0012299945F0700302221B
:2022CB00DFE5114408F511742C75F001F55385F0540222EFE51154F7F511746475F000F529
:2022EB005385F05422740075F000C0E0C0F01207A415811581743C75F000C0E0C0F01227E5
:20230B001A158115817B017C0012299945F0700302234E740775F000C0E0C0F0740175F07B
:20232B0000C0E0C0F012014A1581158115811581744D75F000C0E0C0F01202B31581158124
:20234B0002237B740775F000C0E0C0F0740175F000C0E0C0F012014A1581158115811581C3
:20236B00744175F000C0E0C0F01202B31581158122E511540270030223EF1211D87400751C
:20238B00F000C0E0C0F0740075F000C0E0C0F012014A1581158115811581E56C5403F56C0B
:2023AB00E56C243175F000C0E0C0F01202B315811581742075F000C0E0C0F01202B315811E
:2023CB001581E56C75F000C333C5F033C5F079437A00122888E70987F0C0E0C0F01202DE72
:2023EB001581158122E51154107003022426740075F000C0E0C0F0740175F000C0E0C0F018
:20240B0012014A1581158115811581E5578558F0C0E0C0F01202DE158115812223F42581A6
:20242B00F8868208868308E4FEFF93700122B42555A3E493B42D06430780A3E493B4300377
:20244B0043074024D0B40A00500CCE75F00AA42EFEA3E49380EDE493B46413E60886F0300F
:20246B00F70843072012296FA6F018F68003B4750543070A801CB478054307108014B46FB7
:20248B000B430708800C1226F8A3809BB462624307027A00C004C005C006C007AB075303FE
:2024AB001F7C00E60886F012290DA6F018F6EDD007D006D005D0042430B43A004002240734
:2024CB00C0E00AE645F070CCA902EF30E506742D1226F80A12255DD0E01226F8D9F908080A
:2024EB00EF30E7A5EAC39E50A074201226F80A80F3B4630BAA0112255DE61226F880DFB420
:20250B00732BC082C08386820886837A00E4936004A30A80F8868318868212255DE493A323
:20252B0060051226F880F6D083D08280B1B4691986017A00E76004090A80F912255D860186
:20254B00E7609B1226F80980F7F97A0112255DE980A8EE601B8FF020F716C002EAC39E5053
:20256B000D742030F60274301226F80A80EED002221226887A04C3E637F60809DAF9E4F576
:20258B00F092E0221226887A04C3E697F60809DAF980EB122680C37A04E633F608DAFA8085
:2025AB00DD1226807A04C82AC8C318E613F6DAFA80CC122688AB00A8817F0412287208ACE2
:2025CB0000122631122694A8031225AF5007786DA90412257FA80312263D600CA80412251C
:2025EB00A1A80412263D70DFA803796D1226317FFC022881122688AB00AC011226947D211D
:20260B00C3A8031225A2DD028033786D1225A2786DA90412264C20E7E7786DA904122592B9
:20262B00D380DE1226887A04E7F60908DAFA221226807A0475F000E6700308DAFA22122612
:20264B00887A04E82AF8E92AF9181987F0E6B5F006DAF6E4F5F02274FF40F904F5F00422A4
:20266B00E58124FBF9870012269687000909E7F60809E7F622E58124FBF8860022E5812447
:20268B00FBF886011818860022786D7A04760008DAFB2278FB1228668603088604BB000418
:2026AB00BC00012279E5A3D9FD1BBBFFF01C80F478FB1228668603088604748075F07012FB
:2026CB00290D12296F758921F58DF58B7588597598522278FB1228668682088683E4936014
:2026EB002D1226F8A380F678FB122866E63099FDC299F599B40A17740D80F2E430980C3001
:20270B0098FDC298E599B40D02740A75F0002278FB1228668682088683E075F0002278FB73
:20272B001228668682088683E0F5F0A3E0C5F02278F9122866868208868308E6F02278F91B
:20274B00122866868208868308E608F0A3E6F022D2951227C0C2951227C6C29422C295129D
:20276B0027C0D2952278FB122866E67F0830E704D2958002C2951227C023C294DFEFD2955C
:20278B001227C03095001227C6C2941227C6227F087400D2951227C0A29533C294DFF6C04A
:2027AB00E0D295E571B40002C2951227C0C294D0E075F00022D2943094FD22000022000073
:2027CB0000002278FB1228668601E4FBFCFFE709B42D030FE709C39430B40A005012FA7470
:2027EB000A75F0001228CA2AFBE5F03400FC80E4EB8CF0DF0302296F2278FB122866E6309F
:20280B0099FDC299F5992274FFF5F030980A3098FDC298E59975F0002278FB122866860421
:20282B0018188601E4FD12270AB408028003B47F16ED60F21D74081226F874201226F874E8
:20284B00081226F81980DF1226F8F724F36006090DEDB504D1E4F7F5F0ED22C82581C82265
:20286B00C92581C97A0022D083D082CF2581F581CFC082C08322CF2581F581CF2229F9E590
:20288B00F03AFA227C00CB30E7011CCB2275F00030E70215F022FDE493A3FEE493A3FF4E5E
:2028AB007009E493FE740193FF800BE493A3B5050BE493B5F0068F838E82E473A380D8FE1A
:2028CB00EBA4FD8EF0ECA4FCEB8EF0A4C5F02C2DC5F02212290D8EF0ED22C0F0C0E0E5F06B
:2028EB006C5480FF8CF030F707EB12296FACF0FBD0E0D0F030F70312296FBF800512290DE8
:20290B008062C002C001AAF0F97E007D007F11C3E933F9EA33FADF08F5F0E9D001D00222C0
:20292B00ED33FDEE33FEC3ED9BF5F0EE9C40E0ADF0FED380DBBB000122C333C5F033C5F03C
:20294B00DBF722BB000122C3C5F013C5F013DBF72212295F04700205F02212296814B4FFC2
:20296B000215F022122968F4C5F0F4C5F0221229CC4029801E1229CC40227017801E122935
:20298B00CC40107017800C1229CC501080051229E06009E4F5F0221229E060F7E4F5F00463
:2029AB00221229E040F680EB1229E040EF70E480EB1229E040DD70E480D91229E050DD8078
:2029CB00D2C39BC5F09C20E70720D207C345F02220D2F9D322C5F0C39C7003E5F09B22FB56
:2029EB00E493CB22FCE493FB740193CC22FAE493F9740193CA220A0A4D696E694C4F4747DC
:202A0B0045522056332E3020283F2068656C7029000A3E3E000A0A48454C50204D454E557C
:202A2B00202020202020202020202020202020200A2F207072696E7420616E616C6F672053
:202A4B0072656164696E67202020202020202020202020202020200A742054494D45207331
:202A6B006574202020202020202020202020202020200A64204441544520736574202020FA
:202A8B00202020202020202020202020200A6320436C6F636B20646973706C61792020209C
:202AAB00202020202020202020202020200A73207365742053544152542F53544F502072CD
:202ACB0065636F7264696E672074696D65202020202020202020202020202020200A69203E
:202AEB0073616D706C696E6720496E74657276616C2020202020202020202020202020202B
:202B0B00200A3D20646973706C61792073657474696E6720706172616D657465727320207B
:202B2B0020202020202020202020202020200A72206E756D626572206F66207265636F7275
:202B4B0064202020202020202020202020202020200A62207465726D696E616C20636F6EBE
:202B6B006E656374696F6E202020202020202020202020202020200A6E204E6577207265A1
:202B8B00636F7264202020202020202020202020202020200A6120414C4C20726561643A28
:202BAB002073616D706C65207265616C2D74696D6520616E642064617461202020202020FB
:202BCB00202020202020202020200A78205265616420416C6C3A2073616D706C6520616E88
:202BEB00642064617461202020202020202020202020202020200A752041626F7574204DA5
:202C0B00696E694C4F474745522056332E30202020202020202020202020202020200A3F59
:202C2B002068656C70000A4D696E694C4F474745522077617320646573696E676564206219
:202C4B007920576963686974205349524943484F5445203238204A756E652032303033205D
:202C6B00202020202020202020202020202020200A4170706C69656420506879736963737D
:202C8B0020446570742E204B4D49544C20202020202020202020202020202020200A6669B4
:202CAB00726D7761726520757064617465643A203235204A756E652032303034202020209B
:202CCB00202020202020202020202020200A55524C3A207777772E6B6D69746C2E61632E1E
:202CEB0074682F7E6B7377696368697420656D61696C3A206B73776963686974406B6D6971
:202D0B00746C2E61632E7468000A20312020202032202020203320202020342020202035A3
:202D2B002020202036202020203720202020382020202039202020313020203131202031D6
:202D4B003220202020202020202020202020202020202020200A494E312B20494E312D2084
:202D6B00494E322B20494E322D20494E332B20494E332D20494E342B20494E342D202D3562
:202D8B0056202B35562020305620202B56004D696E694C4F47470045522056332E30000A17
:202DAB00656E7465722063757272656E742074696D652048483A4D4D3A5353203E000A200C
:202DCB00696E74657276616C20312D36303020736563203E20000A656E7465722063757204
:202DEB0072656E7420646174652044442D4D4D2D5952203E000A253032782D253032782D4A
:202E0B00253032782000253032783A253032783A25303278200020256420256420256420DC
:202E2B002564000A2575207265636F72647320617661696C61626C650078302E316D56209D
:202E4B00005265636F72643D20000A535441525420253032643A25303264203E000A5354D4
:202E6B004F502020253032643A25303264203E000A20253032643A253032642025303264B5
:202E8B003A25303264000A20535441525420253032643A25303264000A2053544F5020206A
:202EAB00253032643A25303264000A2053414D504C494E4720494E54455256414C287365ED
:202ECB006329203D202575000A204D414E55414C000A204155544F000A204E6577207265AE
:202EEB00636F72643F28592F4E29000A253032782D253032782D2530327820002530327839
:202F0B003A253032783A2530327820002025640020253032782D253032782D2530327800F4
:202F2B0020253032783A253032783A25303278002025640020256400202564002025640051
:202F4B0020256400202564002025640020256400202564000A3C2D2D20456E7465722064D7
:202F6B0065736372697074696F6E207465787420286D6178203330206368617261637465B5
:082F8B007273292D2D3E0A008E
:00000001FF
